:100000000C9434000C9451000C9451000C94510049
:100010000C9451000C9451000C9451000C9451001C
:100020000C9451000C9451000C9451000C9451000C
:100030000C9451000C9451000C9451000C945100FC
:100040000C9453000C9451000C9451000C945100EA
:100050000C9451000C9451000C9451000C945100DC
:100060000C9451000C94510011241FBECFEFD4E02A
:10007000DEBFCDBF11E0A0E0B1E0ECEFFCE202C0DA
:1000800005900D92A038B107D9F711E0A0E8B1E0D2
:1000900001C01D92A438B107E1F70E9491000C94B1
:1000A0007C160C9400001F920F920FB60F92112431
:1000B0008F939F93AF93BF93809180019091810123
:1000C000A0918201B09183010196A11DB11D809381
:1000D000800190938101A0938201B093830181EE0E
:1000E00086BDBF91AF919F918F910F900FBE0F90E2
:1000F0001F901895F89420918001309181014091D2
:100100008201509183017894B901CA01089514BC09
:1001100083E085BD81EE86BD81E080936E0078949A
:1001200008952F923F924F925F926F927F928F929B
:100130009F92AF92BF92CF92DF92EF92FF920F9376
:100140001F93DF93CF93CDB7DEB7C55ED0400FB618
:10015000F894DEBF0FBECDBF5298539A84B18F631F
:1001600084B98AB1806C8AB987B1837C87B987B139
:10017000807C87B988B1807C88B980E880937A00D8
:1001800080E280937C0080917A00876080937A007F
:1001900080917A00806480937A0014BC83E085BDEE
:1001A00081EE86BD81E080936E007894C353DF4F6B
:1001B0001882CD5CD040C753DF4F188219821A8253
:1001C0001B82C95CD040CB53DF4F188219821A8240
:1001D0001B82C55CD040CF53DF4F188219821A8230
:1001E0001B82C15CD040C354DF4F188219821A822F
:1001F0001B82CD5BD040C754DF4F188219821A8210
:100200001B82C95BD040CB54DF4F188219821A82FF
:100210001B82C55BD040CF54DF4F188219821A82EF
:100220001B82C15BD040C355DF4F188219821A82EE
:100230001B82CD5AD040C455DF4F1882CC5AD040D3
:10024000C555DF4F1882CB5AD040C655DF4F1882B4
:10025000CA5AD040C755DF4F1882C95AD040C85536
:10026000DF4F1882C85AD040C955DF4F1882C75A8D
:10027000D040CA55DF4F1882C65AD040CB55DF4F09
:100280001882C55AD040CC55DF4F1882C45AD0408E
:10029000CD55DF4F1882C35AD040CE55DF4F18825C
:1002A000C25AD040CF55DF4F1882C15AD040C056F5
:1002B000DF4F1882C05AD040C156DF4F1882CF5945
:1002C000D040C256DF4F1882CE59D040C356DF4FC0
:1002D0001882CD59D040C456DF4F1882CC59D04037
:1002E000C556DF4F1882CB59D040C656DF4F188213
:1002F000CA59D040C756DF4F1882C959D040CB5693
:10030000DF4F188219821A821B82C559D040CF56FE
:10031000DF4F188219821A821B82C159D040C357FD
:10032000DF4F188219821A821B82CD58D040C757DE
:10033000DF4F188219821A821B82C958D040CB57CE
:10034000DF4F188219821A821B82C558D040CF57BE
:10035000DF4F188219821A821B82C158D040C358BD
:10036000DF4F188219821A821B82CD57D040ED963A
:100370001CAE1DAE1EAE1FAEED9700EA11E420E0EC
:1003800030E0E9960CAF1DAF2EAF3FAFE997E59691
:100390001CAE1DAE1EAE1FAEE59720ED30E240E074
:1003A00050E0E1962CAF3DAF4EAF5FAFE19788E6EE
:1003B00090E1A0E0B0E0AD968CAF9DAFAEAFBFAF27
:1003C000AD9700EF1AE020E030E0A9960CAF1DAF2A
:1003D0002EAF3FAFA99728E938E040E050E0A5965E
:1003E0002CAF3DAF4EAF5FAFA59780E996E0A0E0A0
:1003F000B0E0A1968CAF9DAFAEAFBFAFA19708E7BD
:1004000015E020E030E06D960CAF1DAF2EAF3FAF92
:100410006D972AE134E040E050E069962CAF3DAFA3
:100420004EAF5FAF699741E050E065965FAF4EAF6A
:10043000659763961CAE1DAE1EAE1FAE63972F96DA
:100440001CAE1DAE1EAE1FAE2F972B961FAE2B9768
:100450002A961FAE2A975FEF29965FAF29978FE7FD
:1004600028968FAF289727961FAE279726968FAF8F
:10047000269725961FAE259724961CAE1DAE1EAE60
:100480001FAE24971CAE1DAE1EAE1FAE18AE19AE29
:100490001AAE1BAE1CAA1DAA1EAA1FAA18AA19AA28
:1004A0001AAA1BAA1CA61DA61EA61FA618A619A638
:1004B0001AA61BA61CA21DA21EA21FA218A219A248
:1004C0001AA21BA21C8E1D8E1E8E1F8E1B8E1A8EB4
:1004D000198E188E1F8A1E8A1D8A5B8B5A8B198A69
:1004E0002F960CAD1DAD2EAD3FAD2F970F5F1F4F5B
:1004F0002F4F3F4F2F960CAF1DAF2EAF3FAF2F9713
:1005000005361105210531050CF401C680917A00EC
:1005100084FFFCCF80917A00806180937A00809183
:1005200079001989143021F42A968FAF2A971BC0BD
:100530002989222321F427968FAF279714C0398960
:10054000333021F428968FAF28970DC04989413068
:1005500021F42B968FAF2B9706C05989523019F48E
:1005600026968FAF26972A968FAD2A97E82FF0E030
:10057000813868F0AFEFB0E0AE1BBF0BFD01E0507B
:10058000FF4FB081B0952996BFAF299706C0E050C4
:10059000FF4F008129960FAF299780917A008064E0
:1005A00080937A0019891F5F198B163008F0198A19
:1005B0008989806280937C002989243039F02F96C4
:1005C0001CAE1DAE1EAE1FAE2F97A1C52B963FAD24
:1005D0002B973295369537703C8B4D9903C061E06F
:1005E00070E002C064E070E04A89473061F45C89E1
:1005F0008B89581741F46596AEADBFAD65976A1704
:100600007B0709F46DC02C892F5F5C895E5F577092
:100610005F5F4C894D5F47704F5F3C893C5F37702F
:100620003F5F9C899B5F97709F5F8C89895F877014
:100630008F5F269FB02D1124C455DF4FB883CC5A4D
:10064000D04027702F5F269F202D1124C555DF4FE6
:100650002883CB5AD040569FE02D1124C655DF4F3A
:10066000E883CA5AD040469FF02D1124C755DF4F6A
:10067000F883C95AD040369F002D1124C855DF4F4A
:100680000883C85AD040969F102D1124C955DF4FBA
:100690001883C75AD040869F202D1124CA55DF4F9A
:1006A0002883C65AD040CB55DF4F5883C55AD04017
:1006B000CC55DF4F4883C45AD040CD55DF4F3883E7
:1006C000C35AD040CE55DF4F9883C25AD040CF5541
:1006D000DF4F8883C15AD04065967FAF6EAF659774
:1006E00028963FAD2897363070F4E996ECACFDAC17
:1006F0000EAD1FADE99755E015950795F794E79472
:100700005A95D1F7FDC128964FAD28974A3038F455
:10071000E996ECACFDAC0EAD1FADE997EAC12896A9
:100720005FAD2897503170F4E996ECACFDAC0EAD9E
:100730001FADE99746E015950795F794E7944A951C
:10074000D1F712C028968FAD28978631F8F4E99634
:10075000ECACFDAC0EAD1FADE99735E015950795F6
:10076000F794E7943A95D1F7E9968CAD9DADAEAD8F
:10077000BFADE99724E0B595A795979587952A95FC
:10078000D1F7E80EF91E0A1F1B1FBAC128969FADAC
:1007900028979C3160F5E996ECACFDAC0EAD1FAD31
:1007A000E997A5E015950795F794E794AA95D1F7F1
:1007B000E9968CAD9DADAEADBFADE997F4E0B595D2
:1007C000A79597958795FA95D1F7E80EF91E0A1F18
:1007D0001B1FE9968CAD9DADAEADBFADE997E6E0D0
:1007E000B595A79597958795EA95D1F7CACF28969D
:1007F000AFAD2897A03238F4E996ECACFDAC0EAD65
:100800001FADE99757C12896BFAD2897B03470F453
:10081000E996ECACFDAC0EAD1FADE99775E0159512
:100820000795F794E7947A95D1F712C02896EFAD23
:100830002897E035D8F4E996ECACFDAC0EAD1FADD1
:10084000E99764E015950795F794E7946A95D1F7D1
:10085000E9968CAD9DADAEADBFADE99753E0B595D2
:10086000A795979587955A95D1F78BCF2896FFAD89
:100870002897F03660F5E996ECACFDAC0EAD1FADF7
:10088000E99744E015950795F794E7944A95D1F7D1
:10089000E9968CAD9DADAEADBFADE99733E0B595B2
:1008A000A795979587953A95D1F7E80EF91E0A1FF7
:1008B0001B1FE9968CAD9DADAEADBFADE99725E0B0
:1008C000B595A795979587952A95D1F75ACF2896EC
:1008D0000FAD2897003738F4E996ECACFDAC0EADBF
:1008E0001FADE997C3C028961FAD289717FD0EC00E
:1008F000E996ECACFDAC0EAD1FADE997B4E01595F3
:100900000795F794E794BA95D1F712C028962FADC2
:1009100028972E38D8F4E996ECACFDAC0EAD1FAD9F
:10092000E997A3E015950795F794E794AA95D1F771
:10093000E9968CAD9DADAEADBFADE997F2E0B59552
:10094000A79597958795FA95D1F71BCF28963FAD38
:100950002897303AF8F4E996ECACFDAC0EAD1FAD3B
:10096000E997E3E015950795F794E794EA95D1F7B1
:10097000E9968CAD9DADAEADBFADE99772E0B59592
:10098000A795979587957A95D1F7E80EF91E0A1FD6
:100990001B1FEACE28964FAD2897423B58F4E996A4
:1009A000ECACFDAC0EAD1FADE99715950795F7942E
:1009B000E794A6C028965FAD2897543B70F4E9965B
:1009C000ECACFDAC0EAD1FADE99754E01595079565
:1009D000F794E7945A95D1F725C028968FAD2897BC
:1009E0008C3B70F4E996ECACFDAC0EAD1FADE99715
:1009F00043E015950795F794E7944A95D1F712C00F
:100A000028969FAD2897943CC0F4E996ECACFDACD9
:100A10000EAD1FADE99732E015950795F794E79471
:100A20003A95D1F7E9968CAD9DADAEADBFADE997E6
:100A3000B595A79597958795A4CE2896AFAD28979D
:100A4000AA3CE0F4E996ECACFDAC0EAD1FADE99725
:100A5000EE0CFF1C001F111FE9962CAD3DAD4EADF5
:100A60005FADE997E20EF31E041F151F82E0159596
:100A70000795F794E7948A95D1F742C028963FAD41
:100A800028973E3CF8F4E996ECACFDAC0EAD1FADFA
:100A9000E997B3E0EE0CFF1C001F111FBA95D1F7C8
:100AA000E9968CAD9DADAEADBFADE997E81AF90AF8
:100AB0000A0B1B0BA3E015950795F794E794AA95ED
:100AC000D1F71EC0E996ECACFDAC0EAD1FADE997B9
:100AD000F4E0EE0CFF1C001F111FFA95D1F7E99608
:100AE0002CAD3DAD4EAD5FADE997E21AF30A040BB4
:100AF000150BE4E015950795F794E794EA95D1F77F
:100B0000C455DF4F9881CC5AD040892F90E0A0E0A7
:100B1000B0E0C652DF4F88839983AA83BB83CA5D46
:100B2000D040C801B701C652DF4F288139814A81C0
:100B30005B81CA5DD0400E943F16C901DA01E1968F
:100B40008CAF9DAFAEAFBFAFE1970A97A105B105DE
:100B500054F42AE030E040E050E0E1962CAF3DAFA5
:100B60004EAF5FAFE197C555DF4F9881CB5AD0406C
:100B7000892F90E0A0E0B0E0CA52DF4F88839983CC
:100B8000AA83BB83C65DD040C801B701CA52DF4FFC
:100B9000288139814A815B81C65DD0400E943F1621
:100BA000C901DA01AD968CAF9DAFAEAFBFAFAD97C7
:100BB0000A97A105B10554F42AE030E040E050E086
:100BC000AD962CAF3DAF4EAF5FAFAD97C655DF4F83
:100BD0009881CA5AD040892F90E0A0E0B0E0CE5270
:100BE000DF4F88839983AA83BB83C25DD040C8014D
:100BF000B701CE52DF4F288139814A815B81C25DC6
:100C0000D0400E943F16C901DA01A9968CAF9DAF72
:100C1000AEAFBFAFA9970A97A105B10554F42AE07A
:100C200030E040E050E0A9962CAF3DAF4EAF5FAF53
:100C3000A997C755DF4F9881C95AD040892F90E0B6
:100C4000A0E0B0E0C253DF4F88839983AA83BB83BF
:100C5000CE5CD040C801B701C253DF4F2881398133
:100C60004A815B81CE5CD0400E943F16C901DA0107
:100C7000A5968CAF9DAFAEAFBFAFA5970A97A10564
:100C8000B10554F42AE030E040E050E0A5962CAFE6
:100C90003DAF4EAF5FAFA597C855DF4F3881C85AFB
:100CA000D040232E332444245524C801B701A20187
:100CB00091010E943F16C901DA01A1968CAF9DAF48
:100CC000AEAFBFAFA1970A97A105B10554F48AE072
:100CD00090E0A0E0B0E0A1968CAF9DAFAEAFBFAF0B
:100CE000A197C955DF4F9881C75AD040692E772404
:100CF00088249924C801B701A40193010E943F16DA
:100D0000C901DA016D968CAF9DAFAEAFBFAF6D97E5
:100D10000A97A105B10554F42AE030E040E050E024
:100D20006D962CAF3DAF4EAF5FAF6D97CA55DF4F9D
:100D30003881C65AD040A32EBB24CC24DD24C80160
:100D4000B701A60195010E943F16C901DA01699613
:100D50008CAF9DAFAEAFBFAF69970A97A105B10544
:100D600054F48AE090E0A0E0B0E069968CAF9DAFCB
:100D7000AEAFBFAF6997E9966CAD7DAD8EAD9FAD5F
:100D8000E997CE52DF4F288139814A815B81C25D6C
:100D9000D0400E943F16C252DF4F2883CE5DD04024
:100DA000C152DF4F3883CF5DD040C052DF4F488300
:100DB000C05ED040CF51DF4F5883C15ED040C25299
:100DC000DF4F088119812A813B81CE5DD040C35716
:100DD000DF4F088319832A833B83CD58D040E9969F
:100DE0006CAD7DAD8EAD9FADE997C253DF4F2881CD
:100DF00039814A815B81CE5CD0400E943F16CE5142
:100E0000DF4F2883C25ED040CD51DF4F3883C35EB1
:100E1000D040CC51DF4F4883C45ED040CB51DF4F30
:100E20005883C55ED040CE51DF4F288139814A8139
:100E30005B81C25ED040C757DF4F288339834A8326
:100E40005B83C958D040E9966CAD7DAD8EAD9FAD4A
:100E5000E997A20191010E943F1619012A01CB577F
:100E6000DF4F288239824A825B82C558D040E9969A
:100E70006CAD7DAD8EAD9FADE997A40193010E944D
:100E80003F1639014A01CF57DF4F688279828A8243
:100E90009B82C158D040E9966CAD7DAD8EAD9FADC3
:100EA000E997A60195010E943F1659016A01C358AE
:100EB000DF4FA882B982CA82DB82CD57D040279605
:100EC0003FAD279737FD02C01D8A06C027964FAD5C
:100ED000279743704E5F4D8BE9966CAD7DAD8EAD1F
:100EE0009FADE997C652DF4F288139814A815B81E6
:100EF000CA5DD0400E943F16C901DA01CB56DF4FD0
:100F000088839983AA83BB83C559D040E9966CAD89
:100F10007DAD8EAD9FADE997CA52DF4F28813981F3
:100F20004A815B81C65DD0400E943F16C901DA014B
:100F3000CF56DF4F88839983AA83BB83C159D040A2
:100F400027965FAD2797252F30E02F773070C901A6
:100F5000880F991F880F991F820F931F880F892F61
:100F6000881F990BA82FAE5FAE8B2696BFAD269734
:100F7000EB2EFF2400E010E0C252DF4F28813981C0
:100F80004A815B81CE5DD0402A5030404040504085
:100F9000A9968CAD9DADAEADBFADA997281B390B01
:100FA0004A0B5B0BC252DF4F288339834A835B8332
:100FB000CE5DD040CA01B901A80197010E94201658
:100FC000272F382F492F552747FD5A952CA73DA786
:100FD0004EA75FA7CE51DF4F88819981AA81BB813F
:100FE000C25ED0400A97A109B109A5962CAD3DADCE
:100FF0004EAD5FADA597821B930BA40BB50BCE51E5
:10100000DF4F88839983AA83BB83C25ED040BC0133
:10101000CD01A80197010E942016272F382F492FB4
:10102000552747FD5A9528A739A74AA75BA786EFFA
:101030009FEFAFEFBFEF280E391E4A1E5B1EA19631
:101040002CAD3DAD4EAD5FADA197221A330A440AD7
:10105000550AC201B101A80197010E942016272F4D
:10106000382F492F552747FD5A952CA33DA34EA352
:101070005FA386EF9FEFAFEFBFEF680E791E8A1E6A
:101080009B1E6D962CAD3DAD4EAD5FAD6D97621A5A
:10109000730A840A950AC401B301A80197010E944A
:1010A0002016272F382F492F552747FD5A9528A35B
:1010B00039A34AA35BA386EF9FEFAFEFBFEFA80E64
:1010C000B91ECA1EDB1E69962CAD3DAD4EAD5FAD9F
:1010D0006997A21AB30AC40AD50AC601B501A801C4
:1010E00097010E942016072F182F292F332727FD3D
:1010F0003A950C8F1D8F2E8F3F8F1C891B8B2F963F
:101100001CAE1DAE1EAE1FAE2F9727E02A8B349962
:1011100004C025961FAE25971EC125963FAD259785
:10112000332329F041E025964FAF259714C1ED9662
:101130008CAD9DADAEADBFADED97CB56DF4F088109
:1011400019812A813B81C559D040801B910BA20B8C
:10115000B30BC753DF4F88839983AA83BB83C95CD2
:10116000D040ED962CAD3DAD4EAD5FADED97CF5679
:10117000DF4F88819981AA81BB81C159D040281B4A
:10118000390B4A0B5B0BCB53DF4F288339834A83E0
:101190005B83C55CD040ED960CAD1DAD2EAD3FAD73
:1011A000ED97C357DF4F88819981AA81BB81CD58C4
:1011B000D040081B190B2A0B3B0B24968CAD9DAD20
:1011C000AEADBFAD2497081B190B2A0B3B0BCF53B9
:1011D000DF4F088319832A833B83C15CD040ED969F
:1011E0000CAD1DAD2EAD3FADED97C757DF4F8881DC
:1011F0009981AA81BB81C958D040081B190B2A0BC1
:101200003B0B8CAD9DADAEADBFAD081B190B2A0BD2
:101210003B0BC354DF4F088319832A833B83CD5B89
:10122000D040ED960CAD1DAD2EAD3FADED97CB573B
:10123000DF4F88819981AA81BB81C558D040081BA6
:10124000190B2A0B3B0B88AD99ADAAADBBAD081BA2
:10125000190B2A0B3B0BC754DF4F088319832A83D2
:101260003B83C95BD040ED960CAD1DAD2EAD3FADBF
:10127000ED97CF57DF4F88819981AA81BB81C158F3
:10128000D040081B190B2A0B3B0B8CA99DA9AEA9BA
:10129000BFA9081B190B2A0B3B0BCB54DF4F08834C
:1012A00019832A833B83C55BD040ED960CAD1DAD01
:1012B0002EAD3FADED97C358DF4F88819981AA814C
:1012C000BB81CD57D040081B190B2A0B3B0BC355D4
:1012D000DF4F088319832A833B83CD5AD04088A9E6
:1012E00099A9AAA9BBA9081B190B2A0B3B0BCF5420
:1012F000DF4F088319832A833B83C15BD040C056EC
:10130000DF4F1882C05AD040C156DF4F1882CF59E4
:10131000D040C256DF4F1882CE59D040C356DF4F5F
:101320001882CD59D040C456DF4F1882CC59D040D6
:10133000C556DF4F1882CB59D040C656DF4F1882B2
:10134000CA59D040C756DF4F1882C959D04091E0E2
:1013500025969FAF2597F894009180011091810107
:101360002091820130918301ED960CAF1DAF2EAF1D
:101370003FAFED9778944A9B3AC5C353DF4F18812E
:10138000CD5CD040112369F063964CAD5DAD6EAD80
:101390007FAD639721E0C353DF4F2883CD5CD040FE
:1013A00071C6CA55DF4F3881C65AD0403150C65633
:1013B000DF4F3883CA59D0405B98ED968CAD9DAD18
:1013C000AEADBFADED97E5960CAD1DAD2EAD3FAD0D
:1013D000E597801B910BA20BB30BE9968CAF9DAFE9
:1013E000AEAFBFAFE99728961FAD2897163050F4DF
:1013F0007C018D01B5E015950795F794E794BA95B2
:10140000D1F7FDC128962FAD28972A3038F4E996F8
:10141000ECACFDAC0EAD1FADE997EAC128963FAD2F
:101420002897303170F4E996ECACFDAC0EAD1FADF1
:10143000E997A6E015950795F794E794AA95D1F753
:1014400012C028964FAD28974631F8F4E996ECACD7
:10145000FDAC0EAD1FADE997F5E015950795F79436
:10146000E794FA95D1F7E9968CAD9DADAEADBFADE1
:10147000E997E4E0B595A79597958795EA95D1F713
:10148000E80EF91E0A1F1B1FBAC128965FAD2897E8
:101490005C3160F5E996ECACFDAC0EAD1FADE997A3
:1014A00075E015950795F794E7947A95D1F7E99645
:1014B0008CAD9DADAEADBFADE99764E0B595A79598
:1014C000979587956A95D1F7E80EF91E0A1F1B1F9D
:1014D000E9968CAD9DADAEADBFADE99756E0B59543
:1014E000A795979587955A95D1F7CACF28968FAD2E
:1014F0002897803238F4E996ECACFDAC0EAD1FAD08
:10150000E99757C128969FAD2897903470F4E996D3
:10151000ECACFDAC0EAD1FADE99745E01595079518
:10152000F794E7944A95D1F712C02896AFAD289763
:10153000A035D8F4E996ECACFDAC0EAD1FADE99743
:1015400034E015950795F794E7943A95D1F7E99625
:101550008CAD9DADAEADBFADE99723E0B595A79538
:10156000979587952A95D1F78BCF2896BFAD289769
:10157000B03660F5E996ECACFDAC0EAD1FADE99769
:10158000F4E015950795F794E794FA95D1F7E99665
:101590008CAD9DADAEADBFADE997E3E0B595A79538
:1015A00097958795EA95D1F7E80EF91E0A1F1B1F3C
:1015B000E9968CAD9DADAEADBFADE99775E0B59543
:1015C000A795979587957A95D1F75ACF2896EFAD3D
:1015D0002897E03738F4E996ECACFDAC0EAD1FADC2
:1015E000E997C3C02896FFAD2897F7FD0EC0E9968E
:1015F000ECACFDAC0EAD1FADE99764E01595079519
:10160000F794E7946A95D1F712C028960FAD289702
:101610000E38D8F4E996ECACFDAC0EAD1FADE997F1
:1016200053E015950795F794E7945A95D1F7E99605
:101630008CAD9DADAEADBFADE99742E0B595A79538
:10164000979587954A95D1F71BCF28961FAD289778
:10165000103AF8F4E996ECACFDAC0EAD1FADE9978D
:1016600033E015950795F794E7943A95D1F7E99605
:101670008CAD9DADAEADBFADE99722E0B595A79518
:10168000979587952A95D1F7E80EF91E0A1F1B1F1B
:10169000EACE28962FAD2897223B58F4E996ECAC79
:1016A000FDAC0EAD1FADE99715950795F794E7943E
:1016B000A6C028963FAD2897343B70F4E996ECAC71
:1016C000FDAC0EAD1FADE997F4E015950795F794C5
:1016D000E794FA95D1F725C028964FAD28974C3B53
:1016E00070F4E996ECACFDAC0EAD1FADE997E3E00C
:1016F00015950795F794E794EA95D1F712C02896C7
:101700005FAD2897543CC0F4E996ECACFDAC0EAD4F
:101710001FADE99772E015950795F794E7947A95D0
:10172000D1F7E9968CAD9DADAEADBFADE997B5955E
:10173000A79597958795A4CE28968FAD28978A3C34
:10174000E0F4E996ECACFDAC0EAD1FADE997EE0C04
:10175000FF1C001F111FE9962CAD3DAD4EAD5FADD6
:10176000E997E20EF31E041F151F42E01595079539
:10177000F794E7944A95D1F742C028963FAD289751
:101780003E3CF8F4E996ECACFDAC0EAD1FADE9972C
:1017900033E0EE0CFF1C001F111F3A95D1F7E996BC
:1017A0008CAD9DADAEADBFADE997E81AF90A0A0B55
:1017B0001B0B23E015950795F794E7942A95D1F72D
:1017C0001EC0E996ECACFDAC0EAD1FADE99794E000
:1017D000EE0CFF1C001F111F9A95D1F7E9962CAD56
:1017E0003DAD4EAD5FADE997E21AF30A040B150B60
:1017F00084E015950795F794E7948A95D1F7C45539
:10180000DF4F9881CC5AD040892F90E0A0E0B0E023
:101810008D879E87AF87B88BC801B7012D853E8520
:101820004F8558890E943F16C901DA01E1968CAFB5
:101830009DAFAEAFBFAFE1970A97A105B10554F4D4
:101840002AE030E040E050E0E1962CAF3DAF4EAFF3
:101850005FAFE197C555DF4F9881CB5AD040892FB4
:1018600090E0A0E0B0E089879A87AB87BC87C80189
:10187000B70129853A854B855C850E943F16C901D1
:10188000DA01AD968CAF9DAFAEAFBFAFAD970A9703
:10189000A105B10554F42AE030E040E050E0AD96F7
:1018A0002CAF3DAF4EAF5FAFAD97C655DF4F9881C0
:1018B000CA5AD040892F90E0A0E0B0E08D839E838B
:1018C000AF83B887C801B7012D813E814F8158850C
:1018D0000E943F16C901DA01A9968CAF9DAFAEAF49
:1018E000BFAFA9970A97A105B10554F42AE030E0EB
:1018F00040E050E0A9962CAF3DAF4EAF5FAFA99747
:10190000C755DF4F9881C95AD040892F90E0A0E099
:10191000B0E089839A83AB83BC83C801B701298176
:101920003A814B815C810E943F16C901DA01A5967C
:101930008CAF9DAFAEAFBFAFA5970A97A105B1051C
:1019400054F42AE030E040E050E0A5962CAF3DAFE3
:101950004EAF5FAFA597C855DF4F3881C85AD0400A
:10196000232E332444245524C801B701A201910138
:101970000E943F16C901DA01A1968CAF9DAFAEAFB0
:10198000BFAFA1970A97A105B10554F48AE090E092
:10199000A0E0B0E0A1968CAF9DAFAEAFBFAFA19776
:1019A000C955DF4F9881C75AD040692E77248824C3
:1019B0009924C801B701A40193010E943F16C901EF
:1019C000DA016D968CAF9DAFAEAFBFAF6D970A9742
:1019D000A105B10554F42AE030E040E050E06D96F6
:1019E0002CAF3DAF4EAF5FAF6D97CA55DF4F38811B
:1019F000C65AD040A32EBB24CC24DD24C801B70195
:101A0000A60195010E943F16C901DA0169968CAFC3
:101A10009DAFAEAFBFAF69970A97A105B10554F46A
:101A20008AE090E0A0E0B0E069968CAF9DAFAEAFE9
:101A3000BFAF6997C455DF4F9881CC5AD0409150C1
:101A4000C056DF4F9883C05AD040C555DF4FA8819C
:101A5000CB5AD040A150C156DF4FA883CF59D040B8
:101A6000C655DF4FB881CA5AD040B150C256DF4F79
:101A7000B883CE59D040C755DF4FE881C95AD0400E
:101A8000E150C356DF4FE883CD59D040C855DF4FF2
:101A9000F881C85AD040F150C456DF4FF883CC5972
:101AA000D040C955DF4F0881C75AD0400150C556B4
:101AB000DF4F0883CB59D040E9966CAD7DAD8EAD3C
:101AC0009FADE9972D853E854F8558890E943F1629
:101AD000C901DA01CB56DF4F88839983AA83BB8380
:101AE000C559D040E9966CAD7DAD8EAD9FADE997FF
:101AF00029853A854B855C850E943F16C901DA012C
:101B0000CF56DF4F88839983AA83BB83C159D040C6
:101B1000E9966CAD7DAD8EAD9FADE9972D813E818F
:101B20004F8158850E943F16C901DA01C357DF4F24
:101B300088839983AA83BB83CD58D040E9966CAD46
:101B40007DAD8EAD9FADE99729813A814B815C8156
:101B50000E943F16C901DA01C757DF4F8883998376
:101B6000AA83BB83C958D040E9966CAD7DAD8EADDC
:101B70009FADE997A20191010E943F16C901DA01C8
:101B8000CB57DF4F88839983AA83BB83C558D04046
:101B9000E9966CAD7DAD8EAD9FADE997A401930143
:101BA0000E943F16C901DA01CF57DF4F888399831E
:101BB000AA83BB83C158D040E9966CAD7DAD8EAD94
:101BC0009FADE997A60195010E943F16C901DA0170
:101BD000C358DF4F88839983AA83BB83CD57D040F6
:101BE000ED962CAD3DAD4EAD5FADED97CB56DF4FD5
:101BF00088819981AA81BB81C559D040281B390BA6
:101C00004A0B5B0BC753DF4F288339834A835B83BF
:101C1000C95CD040ED960CAD1DAD2EAD3FADED973E
:101C2000CF56DF4F88819981AA81BB81C159D040AD
:101C3000081B190B2A0B3B0BCB53DF4F088319836F
:101C40002A833B83C55CD040ED960CAD1DAD2EAD17
:101C50003FADED97C357DF4F88819981AA81BB8142
:101C6000CD58D040081B190B2A0B3B0B24968CAD8A
:101C70009DADAEADBFAD2497081B190B2A0B3B0BD6
:101C8000CF53DF4F088319832A833B83C15CD04045
:101C9000ED960CAD1DAD2EAD3FADED97C757DF4FA7
:101CA00088819981AA81BB81C958D040081B190B32
:101CB0002A0B3B0B8CAD9DADAEADBFAD081B190B18
:101CC0002A0B3B0BC354DF4F088319832A833B83C2
:101CD000CD5BD040ED960CAD1DAD2EAD3FADED977B
:101CE000CB57DF4F88819981AA81BB81C558D040ED
:101CF000081B190B2A0B3B0B88AD99ADAAADBBADE8
:101D0000081B190B2A0B3B0BC754DF4F08831983A1
:101D10002A833B83C95BD040ED960CAD1DAD2EAD43
:101D20003FADED97CF57DF4F88819981AA81BB8165
:101D3000C158D040081B190B2A0B3B0B8CA99DA93D
:101D4000AEA9BFA9081B190B2A0B3B0BCB54DF4FC5
:101D5000088319832A833B83C55BD040ED960CAD85
:101D60001DAD2EAD3FADED97C358DF4F88819981F2
:101D7000AA81BB81CD57D040081B190B2A0B3B0B06
:101D8000C355DF4F088319832A833B83CD5AD04044
:101D900088A999A9AAA9BBA9081B190B2A0B3B0B57
:101DA000CF54DF4F088319832A833B83C15BD04024
:101DB000C656DF4F9881CA59D040C756DF4F988327
:101DC000C959D040ED960CAD1DAD2EAD3FADED9790
:101DD000E5960CAF1DAF2EAF3FAFE597B901A80157
:101DE00011E0C353DF4F1883CD5CD0404BC15B9AE9
:101DF00063964CAD5DAD6EAD7FAD6397E9968CADEE
:101E00009DADAEADBFADE997480F591F6A1F7B1F4F
:101E1000ED960CAD1DAD2EAD3FADED97041715073A
:101E2000260737073CF463964CAD5DAD6EAD7FADD4
:101E3000639723C1C455DF4F1881CC5AD04011504D
:101E4000C056DF4F1883C05AD040C555DF4F288198
:101E5000CB5AD0402150C156DF4F2883CF59D040B4
:101E6000C655DF4F3881CA5AD0403150C256DF4F75
:101E70003883CE59D040C755DF4F8881C95AD040EA
:101E80008150C356DF4F8883CD59D040C855DF4FAE
:101E90009881C85AD0409150C456DF4F9883CC598E
:101EA000D040C955DF4FA881C75AD040A150C55670
:101EB000DF4FA883CB59D040CA55DF4FB881C65AEF
:101EC000D040B150C656DF4FB883CA59D0408A01BE
:101ED0009B01CB56DF4F88819981AA81BB81C5596F
:101EE000D040081B190B2A0B3B0BC753DF4F08834D
:101EF00019832A833B83C95CD0408A019B01CF565A
:101F0000DF4F88819981AA81BB81C159D040081BCC
:101F1000190B2A0B3B0BCB53DF4F088319832A8302
:101F20003B83C55CD0408A019B01C357DF4F88814A
:101F30009981AA81BB81CD58D040081B190B2A0B6F
:101F40003B0B24968CAD9DADAEADBFAD2497081B69
:101F5000190B2A0B3B0BCF53DF4F088319832A83BE
:101F60003B83C15CD0408A019B01C757DF4F88810A
:101F70009981AA81BB81C958D040081B190B2A0B33
:101F80003B0B8CAD9DADAEADBFAD081B190B2A0B45
:101F90003B0BC354DF4F088319832A833B83CD5BFC
:101FA000D0408A019B01CB57DF4F88819981AA815C
:101FB000BB81C558D040081B190B2A0B3B0B88ADC1
:101FC00099ADAAADBBAD081B190B2A0B3B0BC7542F
:101FD000DF4F088319832A833B83C95BD0408A0182
:101FE0009B01CF57DF4F88819981AA81BB81C1585E
:101FF000D040081B190B2A0B3B0B8CA99DA9AEA93D
:10200000BFA9081B190B2A0B3B0BCB54DF4F0883CE
:1020100019832A833B83C55BD0408A019B01C35847
:10202000DF4F88819981AA81BB81CD57D040081BA1
:10203000190B2A0B3B0BC355DF4F088319832A83E7
:102040003B83CD5AD04088A999A9AAA9BBA9081B4E
:10205000190B2A0B3B0BCF54DF4F088319832A83BC
:102060003B83C15BD040C656DF4F9881CA59D040F0
:10207000C756DF4F9883C959D040C353DF4F1882EA
:10208000CD5CD040CB56DF4F88819981AA81BB813E
:10209000C559D040C753DF4F088119812A813B8140
:1020A000C95CD040800F911FA21FB31FED960CADED
:1020B0001DAD2EAD3FADED97081719072A073B0759
:1020C000B4F14C9B2898C056DF4F1881C05AD040BD
:1020D0001F5FC056DF4F1883C05AD040C455DF4F32
:1020E0002881CC5AD040121778F4ED968CAD9DAD76
:1020F000AEADBFADED97C753DF4F88839983AA83F9
:10210000BB83C95CD04013C0ED960CAD1DAD2EADA8
:102110003FADED97C753DF4F088319832A833B8375
:10212000C95CD040C056DF4F1882C05AD040CF564D
:10213000DF4F88819981AA81BB81C159D040CB539F
:10214000DF4F088119812A813B81C55CD040800F17
:10215000911FA21FB31FED960CAD1DAD2EAD3FAD6F
:10216000ED97081719072A073B07B4F14C9B2998EC
:10217000C156DF4F1881CF59D0401F5FC156DF4F86
:102180001883CF59D040C555DF4F2881CB5AD04056
:10219000121778F4ED968CAD9DADAEADBFADED9759
:1021A000CB53DF4F88839983AA83BB83C55CD04020
:1021B00013C0ED960CAD1DAD2EAD3FADED97CB53DD
:1021C000DF4F088319832A833B83C55CD040C15607
:1021D000DF4F1882CF59D040CF53DF4F888199818C
:1021E000AA81BB81C15CD040C357DF4F08811981F0
:1021F0002A813B81CD58D040800F911FA21FB31F71
:1022000024960CAD1DAD2EAD3FAD2497800F911FD0
:10221000A21FB31FED960CAD1DAD2EAD3FADED97DA
:10222000081719072A073B070CF4A5C029961FAD0C
:102230002997812F90E028E030E0CB55DF4FA8812F
:10224000C55AD0402A1B310902C0959587952A9519
:10225000E2F7C256DF4F0880CE59D04002C09595B4
:1022600087950A94E2F780FF02C04C9B2A98C256D9
:10227000DF4FB881CE59D040BF5FC256DF4FB88321
:10228000CE59D040CB55DF4FE881C55AD040BE175C
:1022900030F0C256DF4F1882CE59D0401B8EFE89D7
:1022A000F23098F4ED960CAD1DAD2EAD3FADED972F
:1022B000CF53DF4F088319832A833B83C15CD0400F
:1022C0001CAE1DAE1EAE1FAE56C024968CAD9DAD8D
:1022D000AEADBFAD2497181619061A061B063CF0C2
:1022E00024961CAE1DAE1EAE1FAE249713C02496BE
:1022F0000CAD1DAD2EAD3FAD2497309520951095BA
:1023000001951F4F2F4F3F4F24960CAF1DAF2EAF9F
:102310003FAF24971B8D112351F48CA59DA5AEA52D
:10232000BFA524968CAF9DAFAEAFBFAF24979B8D5A
:102330009F5F9B8FAE899A1780F0ED960CAD1DAD17
:102340002EAD3FADED97CF53DF4F088319832A831E
:102350003B83C15CD0401B8E0EC0ED968CAD9DAD15
:10236000AEADBFADED97CF53DF4F88839983AA837E
:10237000BB83C15CD040C757DF4F88819981AA8158
:10238000BB81C958D040C354DF4F088119812A81CD
:102390003B81CD5BD040800F911FA21FB31F0CADBE
:1023A0001DAD2EAD3FAD800F911FA21FB31FED9647
:1023B0000CAD1DAD2EAD3FADED97081719072A07DF
:1023C0003B070CF49BC029961FAD2997812F90E005
:1023D00028E030E0CC55DF4FA881C45AD0402A1BFA
:1023E000310902C0959587952A95E2F7C356DF4FCC
:1023F0000880CD59D04002C0959587950A94E2F7A0
:1024000080FF02C04C9B2B98C356DF4FB881CD593B
:10241000D040BF5FC356DF4FB883CD59D040CC55B5
:10242000DF4FE881C45AD040BE1730F0C356DF4FAB
:102430001882CD59D0401A8EFE89F23098F4ED966C
:102440000CAD1DAD2EAD3FADED97C354DF4F0883EE
:1024500019832A833B83CD5BD0401CAE1DAE1EAEDC
:102460001FAE4CC08CAD9DADAEADBFAD18161906FC
:102470001A061B062CF01CAE1DAE1EAE1FAE0FC002
:102480000CAD1DAD2EAD3FAD30952095109501954D
:102490001F4F2F4F3F4F0CAF1DAF2EAF3FAF1A8DC9
:1024A000112341F488A599A5AAA5BBA58CAF9DAF22
:1024B000AEAFBFAF9A8D9F5F9A8FAE899A1780F0AB
:1024C000ED960CAD1DAD2EAD3FADED97C354DF4F76
:1024D000088319832A833B83CD5BD0401A8E0EC0BC
:1024E000ED968CAD9DADAEADBFADED97C354DF4F56
:1024F00088839983AA83BB83CD5BD040C754DF4FC9
:1025000088819981AA81BB81C95BD040CB57DF4FBD
:10251000088119812A813B81C558D040800F911FC5
:10252000A21FB31F08AD19AD2AAD3BAD800F911F9F
:10253000A21FB31FED960CAD1DAD2EAD3FADED97B7
:10254000081719072A073B070CF49FC029961FADEF
:102550002997812F90E028E030E0CD55DF4FA8810A
:10256000C35AD0402A1B310902C0959587952A95F8
:10257000E2F7C456DF4F0880CC59D04002C0959591
:1025800087950A94E2F780FF02C04C9B2C98C456B2
:10259000DF4FB881CC59D040BF5FC456DF4FB883FE
:1025A000CC59D040CD55DF4FE881C35AD040BE173B
:1025B00030F0C456DF4F1882CC59D040198EFE89B6
:1025C000F23098F4ED960CAD1DAD2EAD3FADED970C
:1025D000C754DF4F088319832A833B83C95BD040EC
:1025E00018AE19AE1AAE1BAE50C088AD99ADAAADEB
:1025F000BBAD181619061A061B062CF018AE19AE3C
:102600001AAE1BAE13C0998DAD899A1778F008AD3C
:1026100019AD2AAD3BAD30952095109501951F4F12
:102620002F4F3F4F08AF19AF2AAF3BAF198D112382
:1026300041F48CA19DA1AEA1BFA188AF99AFAAAF73
:10264000BBAF998D9F5F998FAE899A1780F0ED96F9
:102650000CAD1DAD2EAD3FADED97C754DF4F0883D8
:1026600019832A833B83C95BD040198E0EC0ED9637
:102670008CAD9DADAEADBFADED97C754DF4F888338
:102680009983AA83BB83C95BD040CB54DF4F888139
:102690009981AA81BB81C55BD040CF57DF4F0881AC
:1026A00019812A813B81C158D040800F911FA21F00
:1026B000B31F0CA91DA92EA93FA9800F911FA21F0E
:1026C000B31FED960CAD1DAD2EAD3FADED970817C8
:1026D00019072A073B070CF49FC029961FAD2997BD
:1026E000812F90E028E030E0CE55DF4FA881C25A1C
:1026F000D0402A1B310902C0959587952A95E2F7AB
:10270000C556DF4F0880CB59D04002C095958795BC
:102710000A94E2F780FF02C04C9B2D98C556DF4F0C
:10272000B881CB59D040BF5FC556DF4FB883CB5976
:10273000D040CE55DF4FE881C25AD040BE1730F0AE
:10274000C556DF4F1882CB59D040188EFE89F23023
:1027500098F4ED960CAD1DAD2EAD3FADED97CB547D
:10276000DF4F088319832A833B83C55BD0401CAAB3
:102770001DAA1EAA1FAA50C08CA99DA9AEA9BFA9B7
:10278000181619061A061B062CF01CAA1DAA1EAA4A
:102790001FAA13C0988DAD899A1778F00CA91DA9AE
:1027A0002EA93FA930952095109501951F4F2F4FC9
:1027B0003F4F0CAB1DAB2EAB3FAB188D112341F43B
:1027C00088A199A1AAA1BBA18CAB9DABAEABBFABBD
:1027D000988D9F5F988FAE899A1780F0ED960CAD1B
:1027E0001DAD2EAD3FADED97CB54DF4F0883198360
:1027F0002A833B83C55BD040188E0EC0ED968CAD0E
:102800009DADAEADBFADED97CB54DF4F88839983BF
:10281000AA83BB83C55BD040CF54DF4F88819981A9
:10282000AA81BB81C15BD040C358DF4F08811981A9
:102830002A813B81CD57D040800F911FA21FB31F2B
:1028400008A919A92AA93BA9800F911FA21FB31F8C
:10285000ED960CAD1DAD2EAD3FADED9708171907E8
:102860002A073B070CF49FC029961FAD2997812F9B
:1028700090E028E030E0CF55DF4FA881C15AD0402A
:102880002A1B310902C0959587952A95E2F7C6560D
:10289000DF4F0880CA59D04002C0959587950A94A9
:1028A000E2F780FF02C04C9B5F98C656DF4FB881AD
:1028B000CA59D040BF5FC656DF4FB883CA59D0400F
:1028C000CF55DF4FE881C15AD040BE1730F0C65611
:1028D000DF4F1882CA59D0401F8AFE89F23098F41F
:1028E000ED960CAD1DAD2EAD3FADED97CF54DF4F46
:1028F000088319832A833B83C15BD04018AA19AA95
:102900001AAA1BAA50C088A999A9AAA9BBA91816D6
:1029100019061A061B062CF018AA19AA1AAA1BAA2D
:1029200013C09F89AD899A1778F008A919A92AA917
:102930003BA930952095109501951F4F2F4F3F4F84
:1029400008AB19AB2AAB3BAB1F89112341F48C8D2B
:102950009D8DAE8DBF8D88AB99ABAAABBBAB9F896C
:102960009F5F9F8BAE899A1780F0ED960CAD1DADE1
:102970002EAD3FADED97CF54DF4F088319832A83E7
:102980003B83C15BD0401F8A0EC0ED968CAD9DADE0
:10299000AEADBFADED97CF54DF4F88839983AA8347
:1029A000BB83C15BD040C358DF4F88819981AA8126
:1029B000BB81CD57D040C355DF4F088119812A8193
:1029C0003B81CD5AD040800F911FA21FB31FED96BF
:1029D0000CAD1DAD2EAD3FADED97081719072A07B9
:1029E0003B07B4F14C9B5E98C756DF4F1881C9591D
:1029F000D0401F5FC756DF4F1883C959D040CA5512
:102A0000DF4F2881C65AD040121778F4ED968CAD6E
:102A10009DADAEADBFADED97C355DF4F88839983B4
:102A2000AA83BB83CD5AD04013C0ED960CAD1DAD2B
:102A30002EAD3FADED97C355DF4F088319832A8331
:102A40003B83CD5AD040C756DF4F1882C959D0407A
:102A5000C753DF4F88819981AA81BB81C95CD0406F
:102A6000E1960CAD1DAD2EAD3FADE197800F911FEE
:102A7000A21FB31FED960CAD1DAD2EAD3FADED9772
:102A8000081719072A073B070CF0289ACB53DF4F8A
:102A900088819981AA81BB81C55CD040AD960CAD7F
:102AA0001DAD2EAD3FADAD97800F911FA21FB31F7F
:102AB000ED960CAD1DAD2EAD3FADED970817190786
:102AC0002A073B070CF0299ACF53DF4F8881998161
:102AD000AA81BB81C15CD040A9960CAD1DAD2EADC5
:102AE0003FADA997800F911FA21FB31FED960CADAC
:102AF0001DAD2EAD3FADED97081719072A073B070F
:102B00000CF02A9AC354DF4F88819981AA81BB8136
:102B1000CD5BD040A5960CAD1DAD2EAD3FADA597BC
:102B2000800F911FA21FB31FED960CAD1DAD2EADF2
:102B30003FADED97081719072A073B070CF02B9AB2
:102B4000C754DF4F88819981AA81BB81C95BD0407E
:102B5000A1960CAD1DAD2EAD3FADA197800F911F7D
:102B6000A21FB31FED960CAD1DAD2EAD3FADED9781
:102B7000081719072A073B070CF02C9ACB54DF4F94
:102B800088819981AA81BB81C55BD0406D960CADCF
:102B90001DAD2EAD3FAD6D97800F911FA21FB31FCE
:102BA000ED960CAD1DAD2EAD3FADED970817190795
:102BB0002A073B070CF02D9ACF54DF4F888199816B
:102BC000AA81BB81C15BD04069960CAD1DAD2EAD15
:102BD0003FAD6997800F911FA21FB31FED960CADFB
:102BE0001DAD2EAD3FADED97081719072A073B071E
:102BF0000CF05F9AC355DF4F88819981AA81BB8110
:102C0000CD5AD04069960CAD1DAD2EAD3FAD699744
:102C1000800F911FA21FB31FED960CAD1DAD2EAD01
:102C20003FADED97081719072A073B070CF05E9A8E
:102C300063964CAF5DAF6EAF7FAF63970C9470023D
:102C4000629FD001739FF001829FE00DF11D649F90
:102C5000E00DF11D929FF00D839FF00D749FF00D1C
:102C6000659FF00D9927729FB00DE11DF91F639FBD
:102C7000B00DE11DF91FBD01CF011124089597FB8F
:102C8000092E05260ED057FD04D014D00AD0001C02
:102C900038F450954095309521953F4F4F4F5F4FF9
:102CA0000895F6F790958095709561957F4F8F4FB9
:102CB0009F4F0895A1E21A2EAA1BBB1BFD010DC058
:102CC000AA1FBB1FEE1FFF1FA217B307E407F507DC
:102CD00020F0A21BB30BE40BF50B661F771F881FB8
:102CE000991F1A9469F760957095809590959B014E
:0C2CF000AC01BD01CF010895F894FFCFA6
:102CFC00FFFEFDFBF7EFDFBF7F3F9FCFE7F3F9FC54
:102D0C00FAF5EBD7AF5F6FB7DBEDF6EEDDBB777B9C
:102D1C00BDDEBE7D7E3E5E6E767A7CBCBAB6AE9E65
:102D2C009DADB5B9D9D5CDCBD3E3C7E3F1F81F8FA2
:102D3C00D3E9F4ECB367DCF0E8D8B878746C5C3C9D
:102D4C003A362E1E1D1B170F1B3363C3C6CC66638E
:102D5C00C6C3C5C9D1D2D46A352D5AB4AC562B4B87
:102D6C0096A653939555AA55AA55AA55AA55AA5550
:00000001FF
